:100000006E2864001720031801282220940108306C
:100010008F00232017200318940A971E94018E0C3A
:100020008F0B0928971A8E1323200E080800260824
:10003000840024088417800484130005171B2406F9
:10004000FF3E0800231717081F39003E8D001608D1
:100050000E3E03188D0A231F522823138C000230F2
:10006000642052288900831608148312080869281E
:1000700088008316081555308900AA308900881435
:1000800088184028081169288F018E00FF308E07DC
:10009000031C8F07031C692803308D00E7305220B2
:1000A00046288D01FC3E8C008D09031C5D28FF3025
:1000B00000008C07031858288C0764008D0F572800
:1000C000080003108D0C8C0CFF3E031861280C08EF
:1000D0006928831303138312640008006400851CDD
:1000E000B0286400851C7528712801308F00F43019
:1000F00045206400851C7E28A901752905158316F5
:10010000051105308312A6000130A400543096007A
:100110004030970001203A3C031D8A2801202A3CE8
:10012000031D8A2801203D3C031D8A2801204A3CEA
:10013000031D8A2801203D3C031D8A280120313CF3
:10014000031D8A280120653C031D8A280120A80080
:100150000130890028083820051183160511831203
:1001600001303220A80085158316851183120530D1
:10017000A6000130A40054309600403097000120C2
:10018000413C031DBF280120643C031DBF28012002
:100190002B3C031DBF2801202B3C031DBF28012041
:1001A000543C031DBF2801207E3C031DBF280120B5
:1001B000213C031DBF280120AD00AA0164002A08CC
:1001C0002D02031C74290530A6000130A400543010
:1001D0009600403097000120AC0064002A082802F5
:1001E000031D7229640080302C02031CFE2880301D
:1001F000AC02861783168613831202298613831690
:1002000086138312640040302C02031C0E294030F8
:10021000AC020617831606138312122906138316DF
:1002200006138312640020302C02031C1E29203088
:10023000AC02861683168612831222298612831632
:1002400086128312640010302C02031C2E291030F9
:10025000AC02061683160612831232290612831682
:1002600006128312640008302C02031C3E29083059
:10027000AC028615831686118312422986118316D5
:1002800086118312640004302C02031C4E290430B2
:10029000AC02061583160611831252290611831625
:1002A00006118312640002302C02031C5E29023006
:1002B000AC02861483168610831262298610831678
:1002C00086108312640001302C02031C6D29AC03DC
:1002D0000614831606108312712906108316061061
:1002E0008312B728AA0FDE28B7286400851C792955
:1002F0007529640029080C3C031D7F29A9016400AD
:100300002908003C031DA429061083160610831239
:100310008610831686108312061183160611831227
:100320008611831686118312061283160612831213
:1003300086128316861283120613831606138312FF
:10034000861383168613831264002908013C031D5B
:10035000AD29061483160610831264002908023C96
:10036000031DBA29061083160610831286148316FD
:100370008610831264002908033C031DC7298610D8
:1003800083168610831206158316061183126400E5
:100390002908043C031DD429061183160611831273
:1003A000861583168611831264002908053C031DF7
:1003B000E12986118316861183120616831606120A
:1003C000831264002908063C031DEE2906128316D9
:1003D0000612831286168316861283126400290879
:1003E000073C031DFB29861283168612831206170B
:1003F00083160613831264002908083C031D082A8B
:100400000613831606138312861783168613831228
:1004100064002908093C031D2D2A061483160610C2
:10042000831286148316861083120615831606110E
:1004300083128615831686118312061683160612FA
:1004400083128616831686128312061783160613E6
:1004500083128617831686138312051583160511DA
:1004600083128515831685116400831229080A3CBE
:10047000031D5A2A0610831606108312861083164F
:1004800086108312061183160611831286118316B5
:1004900086118312061283160612831286128316A1
:1004A000861283120613831606138312861383168D
:1004B00086138312640029080B3C031D7F2A06144F
:1004C0008316061083128610831686108312061573
:1004D000831606118312861183168611831206165F
:1004E000831606128312861283168612831206174B
:1004F0008316061383128613831686138312013024
:10050000AB0064001A302B0203188F2A0A304420F3
:100510006400851C8D2AA90A7529AB0F812A051153
:1005200083160511831285118316851164008312C9
:1005300029080A3C031DBC2A0614831606108312E0
:1005400086148316861083120615831606118312ED
:1005500086158316861183120616831606128312D9
:1005600086168316861283120617831606138312C5
:100570008617831686138312640029080B3C031D1B
:10058000E12A06108316061083128614831686103D
:10059000831206118316061183128615831686119F
:1005A000831206128316061283128616831686128B
:1005B0008312061383160613831286178316861377
:1005C00083120130AB0064001A302B020318F12AA9
:1005D0000A3044206400851CEF2AA90A7529AB0F54
:0805E000E32A75296300F22AE9
:02400E00F63F7B
:00000001FF
